:100000000C9420030C9458030C94BF0B0C94BC0B61
:100010000C94BD0B0C94BE0B0C943D030C94BB0BC9
:100020000C943D030C94C10B0C943D030C943D03C4
:100030000C943D030C943D030C943D030C943D0340
:100040000C943D030C943D030C946F0B0C943D03F6
:100050000C943D030C94C00B0C943D030C943D0395
:100060000C943D030C943D030403090416034D0056
:100070006900630072006F00530070006F0072002F
:10008000740014034E0061007600690047006C00A4
:100090006F00760065001201100100000008C01614
:1000A000DF050001010200010902220001010080B8
:1000B0000A090400000103000000092101010001F8
:1000C000221600070581030800640600FF0901A14C
:1000D00001150026FF00750895800900B20201C0D5
:1000E00080C0E0F0F8FCFEFFFEFCF8F0E0C080000D
:1000F0000000000000FFFFFF000000000000000003
:1001000000000081C3E7FFFF7F7FFFFFFF70787C67
:100110003E1F0F070301000000000103C0C0C0C064
:10012000C0C0C0FFFEFCF8F0E0C080010101010189
:100130000101FF7F3F1F0F0703010E1E3E7CF8F0F9
:10014000E0C0800000000080C0000000000081C30B
:10015000E7FFFFFEFEFFFFFF000000000000FFFFC3
:10016000FF0000000000000103070F1F3F7FFF7F1B
:100170003F1F0F070301C0800000000080C0E0F0B7
:10018000F87C3E1F0FFFFFFFFEFEFFFFE7C381006D
:100190000000000080C0E0F0F8FCFEFFC0C0C0C05E
:1001A000C0C0C0000103070F1F3F7F010101010113
:1001B0000101FFFFFF7F7FFFFFE7C3810000000019
:1001C000000301000000000103070F1F3E7C787050
:1001D0007CFEC6C6C6C6C6C6C6C6C6C6FE7C18381F
:1001E000781818181818181818183C3C7CFEC6C641
:1001F00006060C183060C0C0FC7C7CFEC6C6060635
:100200003C3C0606C6C6FE7CC0C0C0CCCCCCCCCC28
:10021000FEFE0C0C0C0CFEFEC0C0C0C0FCFE0606B0
:1002200006C6FE7C3C7CC0C0C0C0FCFEC6C6C6C6BE
:10023000FE7CFEFEC6C606060C0C181830303030A8
:100240007CFEC6C6C6C67C7CC6C6C6C6FE7C7CFE18
:10025000C6C6C6C6FE7E060606067C7800000000FE
:100260000000000000000000000000000044440402
:10027000AA00000AEAEA46C46CA2448A4A4AA6488E
:10028000000024444284444804E4E4004E4000005A
:1002900048000E000000042244884AAAA44C444EA0
:1002A0004A248EC2422C8AAE22E8C22C48CAA4E25A
:1002B00024444A4AA44AA624004040004048024838
:1002C0004200E0E00842484AA4004AEE864AAEAA4C
:1002D000CACAAC4A88A4CAAAACE8C88EE88C884AC4
:1002E0008AA6AAEAAAE4444EE44448AACCAA88888A
:1002F0008EAEEAAAAEAAAA4AAAA4CAAC884AAAE6BC
:10030000CAACCA68422CE44444AAAAA4AAAA44AA31
:10031000AEEAAA44AAAAA444E2448E6444468844AD
:1003200022C4444CA4AAA4A0AAA44200004D2020A8
:10033000200044462020004D4158200041564720CF
:10034000004B4D202000414257200054494D4500AC
:100350004155462000485E48450053504420004423
:10036000495354005452495000414C5420004153C9
:1003700043200044455343000020202000534554AF
:10038000555000545241434B00524F555445005371
:10039000544F500057454954455200434F4E54491D
:1003A0004E554500524553455400545241434B323B
:1003B000524F5554450045494E004F4E004155534C
:1003C000004F464600525F434B574547005741593F
:1003D0004241434B00414B5420485E484500414C4C
:1003E000544954554445004D415820485E48450005
:1003F0004D415820414C54004D41582053504545E3
:1004000044004156205350454544005354524543FF
:100410004B450041424641485254004449535441DF
:100420004E434500444F574E48494C4C00545249A6
:10043000502054494D4500485E48452041554600EE
:10044000415343454E5400485E48452041425700C1
:1004500044455343454E5400444555545343480086
:100460004745524D414E00454E474C495343480085
:10047000454E474C495348004D4554524953434813
:10048000004D455452494300494D50455249414C55
:10049000004D4548520055500057454E494745527A
:1004A00000444F574E0054494D45205554432B00AE
:1004B00046554E4B54494F4E454E0046554E4354BB
:1004C000494F4E530053505241434845004C414E12
:1004D00047554147450045494E4845495400554E0A
:1004E000495453005A454954004B4F4E54524153BE
:1004F0005400434F4E545241535400455849540000
:100500007803550355035A035A035F035F036403DB
:1005100055035503780378037803690369035A0385
:100520005A035F035F036403690369037803780375
:1005300078032D03370337033C03410346034B0382
:1005400050034603780378037803320337033703F5
:100550003C032D0373034B036E037303780378038B
:100560007D0383038903B004C504D604E404E904CD
:10057000FB0400007D0383038903BB04CD04DE0478
:100580004B03F204FB040000B004D503E703F803B7
:1005900002040B0413042D0437044704FB04000079
:1005A000BB04DE03F003F80302041B0424042D043F
:1005B00040045004FB04000083038F039403A4034E
:1005C000AA03FB04000083038F039B03A403AA0375
:1005D000FB0400008903B603BD03A403C503FB04A9
:1005E00000008903BA03C103A403CD03FB04000088
:1005F000C50458046704FB040000CD0460047004C3
:10060000FB040000D60478048804FB040000DE0428
:1006100081048804FB040000A60491049904FB04EF
:100620000000A6049604A104FB040000E904910460
:100630009904FB040000F2049604A104FB040000EA
:1006400011241FBECFEFD4E0DEBFCDBF12E0A0E08B
:10065000B1E0E8EDF6E302C005900D92AC30B107D1
:10066000D9F713E0ACE0B2E001C01D92AE3BB10798
:10067000E1F70E94DB060C946A1B0C94650BA82F13
:10068000B92F80E090E041E050EA60956F5F58F448
:100690002D9138EF82279795879510F0842795271D
:1006A0003F5FC8F3F3CF0895EADF8D939D930895DC
:1006B000CF93CFB7CF93C3954C9BE9F74C9B09C021
:1006C0004C9B07C04C9B05C04C9B03C04C9B01C07E
:1006D000A3C0DF93C0913C02DD27CD5BDD4F4C9B77
:1006E00002C0DF91EBCF2F930F931F9309B12FEF30
:1006F00004FB20F94F933F9319B14FEF012704FBFF
:1007000021F93BE031C04E7F012F19B1216028C093
:10071000102F4D7F2260000009B129C04B7F24605B
:10072000012F000019B12BC019B1477F28602AC0E2
:100730004F7E09B120612CC04F7D19B120622FC0BE
:100740004F7B09B1206432C0422709B149934FEF72
:100750000000102714FB20F919B11471C9F1297F89
:1007600091F2012704FB21F909B1237F89F231506D
:1007700058F1102714FB22F919B1277E79F20127CD
:1007800004FB23F92F7C81F209B1102714FB24F913
:100790002F7971F200C019B1012704FB25F92F73DD
:1007A00059F200C009B1102714FB26F9223040F29B
:1007B00000C019B1012704FB27F9243028F64F7730
:1007C000206819B10000F9CF11E01CBB002719C047
:1007D0003B503195C31BD04011E01CBB0881033C4A
:1007E000F9F00B34E9F020913A021981110F12133C
:1007F000EDCF4A81441F093641F10D3211F0013E1F
:1008000029F7009341023F914F911F910F912F9132
:10081000DF91CCB3C0FD4FCFCF91CFBFCF91189513
:1008200020914102222379F310913F02112369F5AF
:1008300034306AF130933F0220933B0210913C0226
:100840003BE0311B30933C0222C000913F0201305B
:10085000E4F40AE54F7049F43091000134FD19C009
:1008600000930001C3E2D2E018C030912E0234FDA3
:1008700010C000932E02CFE2D2E00FC02795A8F45B
:100880005150A9F4220F0000F9CF4AE503C042ED10
:1008900001C0432FC4E1D0E032E01AB114615C9A88
:1008A0001AB90BB120E414E15F93012756E00BB9AC
:1008B000279520F4515021F4220FF9CF012756E05B
:1008C00000003B5A0BB9D0F2279528F4515029F477
:1008D000220F0000F9CF012756E027950BB920F42D
:1008E000515021F4220FF9CF012756E029913323EB
:1008F0000BB921F60B7E10914002110FC651D0406A
:100900000BB911F010933A0211E01CBB00611AB14F
:100910001B7E402F4B7E5F9100C000C00BB91AB9FF
:100920004BB971CFE9E6F0E0808182608083E89A7C
:100930008BE480932F028AE580932E0208951F9303
:10094000CF93DF9360913F02635067FDBFC08091FA
:100950003C02CCE0D0E0C81BD109CD5BDD4F8091DB
:100960003B028D3209F09FC0683009F0ADC083ECC6
:10097000809323028AE58093000110920C02888103
:10098000807641F0CE010E942206282F8F3F09F485
:1009900079C07FC09A8110922C028981882321F42A
:1009A00010922D0222E067C0853019F49093400226
:1009B00061C0863009F04AC08B81813041F486E9FC
:1009C00090E090933E0280933D0222E13BC0823052
:1009D00041F488EA90E090933E0280933D0222E247
:1009E00031C08330D1F48A81882341F488E690E0D5
:1009F00090933E0280933D0224E024C0813019F49C
:100A00008CE690E018C08230E1F482E890E09093A8
:100A10003E0280933D0224E115C0813241F48AEB0D
:100A200090E090933E0280933D0229E00BC0823219
:100A300041F48AEC90E090933E0280933D0226E1DF
:100A400001C020E080E480930C0223C0883021F4B0
:100A500021E082E492E011C0893019F490934202BF
:100A600009C08A3011F421E006C08B3019F48BE400
:100A700080932F0220E08CE292E090933E028093DC
:100A80003D0207C0888187FD2E8180E880930C029B
:100A900006C08F81882319F48E81821708F0822F77
:100AA0008093010111C080910C0287FF0DC0CE011F
:100AB0000E942A088F3F21F48EE18093000104C038
:100AC000882311F01092010110923F0280910001E1
:100AD00084FF5AC0809101018F3F09F455C0182F3F
:100AE000893008F018E0811B809301018091230276
:100AF00098E8892780932302112399F180910C02B1
:100B000087FF09C084E292E0612F0E94E808182F55
:100B10008930A0F526C020913D0230913E0286FF2B
:100B20000DC0A4E2B2E080E090E0F901E80FF91F07
:100B3000E491ED9301961817C1F708C0D901912FE0
:100B4000E4E2F2E08D9181939150E1F71150812F11
:100B500090E01F5F0196820F931F90933E02809357
:100B60003D0284E292E0612F0E945403612F6C5F8A
:100B70006C3041F08FEF8093010104C08FEF8093C0
:100B800001016EE16093000194E189B1847131F457
:100B90009150D9F71092400210923A02DF91CF9112
:100BA0001F91089580916102882309F04AC086B19F
:100BB00080958370833009F444C090911502913080
:100BC000A1F0913018F09230D9F534C08823C1F1EA
:100BD0008093160281FF02C082E003C080FF03C041
:100BE00083E08093610281E01CC0882329F1909109
:100BF0001602923061F4809114028F31A8F082E8DD
:100C000080936102909315021092140219C09130E2
:100C100059F4809114028F3138F083E88093610297
:100C200082E080931502F0CF809114028F5F809351
:100C3000140206C0882321F41092160210921502A5
:100C4000A8950895FC0180818076803261F48181CD
:100C5000813011F0893039F480E8809318021092C5
:100C600017028FEF089580E008958091620281302D
:100C700029F08130C0F08230A1F408C05B9A84E092
:100C80008093120282E080936202089580911202A2
:100C90008150809312028F5F31F45B981092620250
:100CA000089510926202089580910F028230B9F087
:100CB000833038F4882309F47DC0813009F078C08E
:100CC00006C0833079F1843009F072C03CC0809353
:100CD00062025B9A84E08093130282E031C08091CB
:100CE00013028150809313028F5F09F063C05B98F9
:100CF0008091EF029091F0026FE070E00E949F1AE5
:100D0000CB01880F991F63E80E9421196091EF02BF
:100D10007091F00282E090E00E94551B0E948509CC
:100D200083E00EC086B190E08095909583709070BE
:100D3000892B09F03FC05D988AE08093130284E01C
:100D400080930F02089580911302815080931302C3
:100D50008F5F81F585E20E94670914BE88E10FB6B6
:100D6000F89480936000109260000FBE1DBA92E06C
:100D700090936C0087E08BBB909368008FEE80931C
:100D8000640083B7817F846083BF83B7816083BF42
:100D9000889583B78E7F83BF2BE088E190E00FB604
:100DA000F894A895809360000FBE20936000FFCF59
:100DB00010920F0208952EE088E190E00FB6F894AB
:100DC000A895809360000FBE209360000E94C20B24
:100DD0000E94EB0B0E949204549A20E048E95AE3E7
:100DE00004C0CA010197F1F7A8952150D1F7549892
:100DF000789481E090E00E94391B8093FB028F5031
:100E0000813718F08CE38093FB020E94980982E0FE
:100E100090E00E94411B9093F0028093EF028AE0E1
:100E200090E00E94411B90935E0280935D0280E0FF
:100E300090E00E94391B8093EE0290E083709070E6
:100E4000892B19F081E090E802C082E090E890934D
:100E5000010380930003909305038093040384E0CF
:100E600090E00E94411B90933801809337018F5F7F
:100E70009F4F31F485E590E09093380180933701DE
:100E800081E0809360022DEC32E13093F8022093F0
:100E9000F70280936102809306038EEF80936602CF
:100EA000EE24FF2400E010E0CC24C39474E6A72EC7
:100EB00065E0762E53E0852E44E0D42E39E0932E63
:100EC0000E949F0480910B038111FF2480910B03EA
:100ED000882341F080910E02882321F410920B03A5
:100EE0000E947C14183C10F41F5F7DC080910E029C
:100EF000DA9B08C0DBBA882311F4D0926102C09259
:100F00000E0206C0813011F4D092610210920E02DE
:100F10000233D0F184E08F1510F0F39403C0C09237
:100F20006202FF2480917A0084FF92C020917800B1
:100F30003091790083E02132380720F480910E024D
:100F4000882319F07092660283C082E02D3B380737
:100F500018F0D09266027CC082E02B38380718F077
:100F60008092660275C082E02D36380720F082E05C
:100F7000809366026DC02F54324018F0C092660212
:100F800067C01092660264C00F5F013329F480913C
:100F90007A00806480937A0080910603873071F430
:100FA000809167038A9DC001112420918603820FDE
:100FB000911D62E042E02CE30E94AF0C802F90E094
:100FC00083709070892B51F40E94D2058091610248
:100FD000823821F4C0920F02109261020E945406DE
:100FE0000E94350610E0E39401F5B39471F480910A
:100FF000F7029091F8028D5C924139F48091600281
:1010000084FD03C082E08093610280910201882305
:1010100021F081508093020108C0809161028823F1
:1010200021F490926102A092020180910F02882324
:1010300059F4E091F702F091F8028091610209956C
:10104000809361028823A9F7B99BFECFB99A38CF64
:1010500000E0A2CF1F93482F792F80911802162FFE
:10106000861708F4182F2091170230E027593D4FBA
:10107000C901642F412F50E00E94281B9091170254
:10108000910F9093170280911802811B8093180290
:1010900020916902273419F4943038F004C02434C4
:1010A00021F4933010F010921802809118028823D6
:1010B00009F085C0209310022734B1F590916A029F
:1010C0009C3FD9F09D3F18F49B3F39F51AC09D3FD6
:1010D000C1F09E3F11F583E080930D028091EF02F5
:1010E0009091F0026FE070E00E949F1ACB01880F90
:1010F000991F63E80E94211962C082E080930D026B
:101100005EC081E090E09093300180932F011092B7
:101110000D0281E08093610252C080916B02809346
:101120005B0290935C024BC0253409F580916B0201
:1011300080935D0280916A0280935E0280916D02CD
:101140008093670280916C028093680260915D02D7
:1011500070915E028AE090E00E94551B6091EF0260
:101160007091F00282E090E00E94551B28C020356B
:1011700031F590916A029C3F49F481E080930D0221
:10118000809160028E7F8093600219C09B3F49F47A
:1011900010920D0281E090E09093300180932F0136
:1011A0000EC080916B0280935B0290935C02609111
:1011B0005B0270915C028CE692E00E943E1990E026
:1011C00080911802882309F491E0892F1F910895D6
:1011D000FF920F931F93082FF92E462F8091110233
:1011E000861710F46093110280911802142F84174F
:1011F00008F4182F80911702882309F04DC081E070
:101200008093630280911002873491F460915B02B5
:1012100070915C0289E692E00E942D1A80915B0237
:1012200090915C02019690935C0280935B0234C0C3
:10123000833581F5809369028AE380936A02109274
:101240006C0210926B0280915D0290915E0290930D
:101250006E0280936D0288E592E090937002809315
:101260006F028091EF029091F0029093720280934E
:1012700071028091590290915A0290937402809366
:101280007302809160028093750280910D028093B9
:10129000760202C0109263022091170230E02759B3
:1012A0003D4F802F9F2DB901412F50E00E94281BF8
:1012B00080911702810F8093170280911802811B81
:1012C00080931802812F1F910F91FF9008952A9803
:1012D00029988EBD0DB407FEFDCF2A9A08952A984D
:1012E000299A8EBD0DB407FEFDCF2A9A08951F934B
:1012F000162F95E0981B892F80640E946709812F23
:1013000080680E9467091F91089585E060E00E944F
:1013100077092A98299A80E090E01EBC0DB407FE58
:10132000FDCF019621E0883F9207B9F72A9A0895E8
:10133000289A2898289A80E58CBD2A9A81E20E94F2
:10134000670988EC0E94670986E00E94670983E1CB
:101350000E9467098091FB0280680E94670980E211
:101360000E9467098CE00E9467090E948509089520
:10137000AF92BF92DF92EF92FF920F931F93CF93A2
:10138000DF93182F062FD42E8052803408F045C0EA
:1013900081E0481719F48FEF0E946F0923E0129F34
:1013A000C00111243AE0E32E32E0F32EE80EF91EDC
:1013B000029FE0011124C65FDD4F2DE0A22E22E046
:1013C000B22EA80EB91EF7010491FE011491912FBF
:1013D00092959F70802F807F982BF1E0DF1609F4A3
:1013E0009095892F0E946F09802F8295807F1F70B2
:1013F000812B91E0D91609F480950E946F09089419
:10140000E11CF11C2196EA14FB04E9F6DD2011F041
:101410008FEF01C080E00E946F09DF91CF911F9193
:101420000F91FF90EF90DF90BF90AF900895FF92E3
:101430000F931F93CF93DF93EC01162FF42E022FFF
:1014400011C0812F6F2D0E947709888169816623E1
:1014500009F460E2402F0E94B8098981882329F0AD
:1014600022961F5F8881882361F7DF91CF911F91BA
:101470000F91FF900895DF92EF92FF920F931F93C9
:10148000CF93DF93EC01062FD42EE22E15C0802FD0
:101490006D2D0E9477092196FE0114912197112349
:1014A00011F460E201C0612F8F2D4E2D0E94B8090A
:1014B000112331F022960F5FFE01F490FF2039F7DF
:1014C000DF91CF911F910F91FF90EF90DF900895E2
:1014D0000F931F93CF93DF93182F862F022F642F24
:1014E0000E9477091A3008F01AE08EE0189FE00198
:1014F0001124C053DE4F10E0FE018491002319F047
:101500001D3009F481600E946F091F5F21961E3013
:1015100099F7002329F081E00E946F0981E001C062
:1015200080E00E946F09DF91CF911F910F91089584
:101530008F929F92AF92BF92CF92DF92EF92FF92E3
:101540000F931F93CF93DF93182F962E842E862F01
:10155000642F0E9477091A3008F01AE08EE0189F75
:1015600060011124AA24BB24B39480ED91E0C80E3D
:10157000D91E2FC0FE01949196959695892F8B21A7
:1015800011F410E001C01FE0F2E0AF1639F0892F2E
:1015900090E08E219F21892B09F0106F812F0E94EE
:1015A0006F09812F0E946F09812F0E946F09812F7F
:1015B0000E946F090F5F21960E30E1F69A94892DF3
:1015C000682D0E947709A39483E0A81649F0BB0C0C
:1015D000BB0CEB2CFF24EE0CFF1CE60100E0CACF95
:1015E000DF91CF911F910F91FF90EF90DF90CF90FF
:1015F000BF90AF909F908F900895EF92FF920F93BE
:101600001F93E62EF42E082F0CC0802F6F2D0E9402
:10161000770910E080E00E946F091F5F1031D1F759
:101620000F5FE01690F71F910F91FF90EF900895D4
:10163000FF920F931F93CF93DF93182F8091030195
:10164000181709F43CC010930301183020F08FEFF5
:101650008093030134C083E06FE00E947709110F8B
:10166000012F10E0E80164E0CC0FDD1F6A95E1F77F
:10167000C01BD10BC052DF4FFF24FE0184910E949A
:101680006F09F3942196FFE0FF16B9F782E06FE04F
:101690000E947709C8010196EC0154E0CC0FDD1FD0
:1016A0005A95E1F7C81BD90BC052DF4F10E0FE017D
:1016B00084910E946F091F5F21961F30C1F7DF914F
:1016C000CF911F910F91FF9008951F920F920FB627
:1016D0000F9211240F900FBE0F901F9018951F921C
:1016E0000F920FB60F9211248F939F93EF93FF9356
:1016F0009091C60080911902813079F0813018F004
:10170000823071F526C0943269F581E08093190228
:1017100010921A0290930C0325C0943209F1E091C3
:101720001A029A3261F0EF5FE0931A02E83510F086
:1017300010921902F0E0E45FFC4F908313C0F0E0D8
:10174000E45FFC4F118280930B0382E080931902C7
:1017500009C080910B03882329F41092190202C05A
:1017600010920B03FF91EF919F918F910F900FBEFD
:101770000F901F901895189518951895189518950D
:10178000189518958FEE84B980E185B98CE787B9F3
:1017900087E088B98AEE8AB91BB85D9A84E18093A4
:1017A0006D00E1E6F0E090E8908310829093640091
:1017B00087EC80937C0086E880937A0082E08093B7
:1017C000B0008093B10086E98093B30090BF1DBA4A
:1017D0001092700008951092C5008CE08093C400B0
:1017E00080E98093C1008EE08093C200089581302B
:1017F00021F483E08093EE020895823011F4109278
:10180000EE020895813031F4809149018C305CF40E
:101810008F5F07C0823039F480914901853F1CF009
:1018200081508093490180E090E29093340180934D
:1018300033010895682F8091EE0281FD08C08FE189
:10184000689FC001112462E370E00E949F1A862FF6
:1018500008952EE731E0281B390B81E0293638073F
:1018600010F028563140C9016DE270E00E949F1AC5
:10187000862F8A5F883008F088500895CF93DF93D1
:10188000EB01FC01F695E795282F2170205DCF0133
:1018900065E070E00E949F1A880F991F280F288327
:1018A0002197CF0165E070E00E949F1ACB0161157E
:1018B000710539F7DF91CF91089520E32093F1026C
:1018C0002093F2022093F3022093F4022093F50276
:1018D00065EF72E00E943E0C08950F931F93162F40
:1018E000042F0E945D0C8091F202803319F480E293
:1018F0008093F202812F602F0E9477098091F2027B
:101900006091F30240E00E94B809812F8F5F602F41
:101910000E9477098091F4026091F50240E00E94F4
:10192000B8091F910F9108951F93109189031A30E0
:1019300008F019E084E060E00E94770983E561E443
:1019400040E00E94B80985E060E00E947709105DE0
:1019500084E5612F40E00E94B8091F910895EF923D
:10196000FF920F931F93CF93DF93382F592FF42EAD
:10197000E22E8AE08093F1028093F2028093F302D8
:1019800080E38093F4021092F502062F643008F091
:1019900003E0902F9F5F83E020E3E82FF0E0EF501B
:1019A000FD4F2083915081509923B9F7832F952FB4
:1019B0009C0187E22031380710F02FE037E2C9019F
:1019C00064EF72E00E943E0C14E0101BC1EFD2E005
:1019D00019C0982F9053115021968881882341F087
:1019E00020E0112309F421E0892F6F2D4E2D04C032
:1019F000892F6F2D4E2D20E00E94680AF39485E018
:101A00008F1518F08881882321F7DF91CF911F91DE
:101A10000F91FF90EF9008959C018091EE0281FD5F
:101A20000BC0C90155E0880F991F5A95E1F762E68E
:101A300070E00E949F1A9B01C90160E042E02CE324
:101A40000E94AF0C089582E065E04AE20E94FD0A20
:101A5000809168030E941A0C90E060E042E02AE264
:101A60000E94AF0C0895DF93CF93CDB7DEB72997CF
:101A70000FB6F894DEBF0FBECDBF20917C03822F3E
:101A80006AE00E94931A805D8983822F0E94931AD4
:101A9000905D9A838AE38B8320917D03822F0E943D
:101AA000931A805D8C83822F0E94931A905D9D8390
:101AB0008EE28E8320917E03822F0E94931A805D96
:101AC0008F83822F0E94931A905D98871986CE018A
:101AD000019662E04DE420E00E94170A29960FB6B5
:101AE000F894DEBF0FBECDBFCF91DF9108958091F6
:101AF0000E02882391F184E091E060E040E020E074
:101B00000E94170A80910D02813029F480915B02B6
:101B100090915C0243C0823079F420915B02309155
:101B20005C0236952795C901E4E0880F991FEA9574
:101B3000E1F7821B930B32C08330E1F520915B0209
:101B400030915C0236952795C90164E0880F991F92
:101B50006A95E1F7821B930B1FC08091600281FFA1
:101B60000CC08FE091E060E040E020E00E94170AA6
:101B70008091590290915A0211C08091600280FFB9
:101B800012C085E191E060E040E020E00E94170A89
:101B90008091EF029091F0028855924060E040E21F
:101BA0000E946D0C08958BE191E060E040E020E040
:101BB0000E94170A8AE091E060E040E220E00E9483
:101BC000170A08958091EE0281FF03C081E291E03F
:101BD00002C086E291E060E04AE220E00E94170A3B
:101BE0000E94940C0E94330D0E94230D0E94770DD9
:101BF00008951F9381E06CE40E94770980E260E21F
:101C000040E00E94B80980E06CE40E94770980916E
:101C100066028E3F41F48BE291E060E04DE420E00B
:101C20000E94170A14C08CE30E946F098FEF0E9474
:101C30006F0915E080916602811710F08FEF01C0E7
:101C400081E80E946F09112311F01150F3CF1F9109
:101C50000895482F82FF03C081E08093060341FF6F
:101C600031C080913701909138019F70892B31F4F8
:101C700082E090E0909338018093370160913701C2
:101C80007091380120910603A1E0B0E02F5FE22FB0
:101C9000F0E0EE0FFF1FE857FA4F85919491892BE2
:101CA00009F421E0822F90E00197FD0102C0EE0FC0
:101CB000FF1F8A95E2F7CF0186239723892B31F303
:101CC0002093060340FF4BC00E94F90D82E065E0BF
:101CD0004CE30E94FD0A8091EE029091060380FF82
:101CE00009C0E92FF0E0EE0FFF1FE050FB4F6591B8
:101CF000749108C0E92FF0E0EE0FFF1FE85EFA4F85
:101D00006591749181EF92E00E94211B81EF92E036
:101D100060E04CE320E00E94170A8091EE0290916F
:101D2000060381FF09C0E92FF0E0EE0FFF1FE05D21
:101D3000FA4F6591749108C0E92FF0E0EE0FFF1F94
:101D4000E85BFA4F6591749181EF92E00E94211B4C
:101D500081EF92E060E044E420E00E94170A809165
:101D60000603853059F1863060F48230C1F083304B
:101D700018F48130F1F50EC08330B1F08430C9F52C
:101D800018C08730E9F18730F0F0883031F18930C0
:101D900081F528C0809182039091830327C08091B0
:101DA00087039091880322C08091930390E060E0C4
:101DB0000FC0809194039091950309C080918C038A
:101DC00090918D0304C08091690390916A0361E052
:101DD00042E02CE30E94AF0C089580918A03909119
:101DE0008B0304C080919103909192030E940C0D8B
:101DF000089580E090E060E042E02CE30E94AF0CA8
:101E000008951F93809168030E941A0C182F84363E
:101E100008F013E6812F6AE00E94931A892F65E08B
:101E200040E00E94980A812F6AE00E94931A62E0C3
:101E300040E00E94980A1F9108956F927F928F92BE
:101E40009F92AF92BF92DF92EF92FF920F931F93F8
:101E5000CF93DF935C014B01D42E0E948509F501DD
:101E60008591949160E040E020E00E943B0A88E088
:101E70008D1518F0FF24F39403C079EFF72EFD0CB5
:101E80006DE0E62E51E0652E712CCF2DD0E0FE01E5
:101E9000EE0FFF1FEA0DFB1D0591149101151105B1
:101EA00089F180E06E2D0E9477092197C30102C05D
:101EB000880F991FCA95E2F788219921892B41F053
:101EC000F801649140E0FD1409F441E08BE207C0A1
:101ED000F801649140E0FD1409F441E080E20E94C1
:101EE000B809C801019620E0FD1409F421E061E081
:101EF0004E2D0E943B0AFCE4EF1621F089E0E80E2B
:101F0000F394C3CFDF91CF911F910F91FF90EF908A
:101F1000DF90BF90AF909F908F907F906F900895CB
:101F20001F93182F833009F47EC0843030F4813041
:101F300051F0823009F0BDC05FC0843041F0833879
:101F400009F0B7C0AEC00E94850910934701E09127
:101F50000703F0910803608171818091FC029091E8
:101F6000FD02409147010E941D0FE0910703F0918F
:101F700008030190F081E02DE070F07780E1E0301F
:101F8000F80721F48091FB0290E031C080E2E0305C
:101F9000F80719F580914901992787FD909597FFDA
:101FA00003C0909581959F4F64E040E00E946D0CC6
:101FB00080914901181614F41BE205C0882311F022
:101FC0001DE201C010E284E060E00E94770980E237
:101FD000612F40E00E94B8096CC0E050F04309F066
:101FE00068C08091EF029091F0028855924064E0C1
:101FF00040E00E946D0C5DC0809147018F5F80932F
:10200000470190E0880F991FE091FC02F091FD02DA
:10201000E80FF91F85919491892B09F040C081E068
:10202000809347013CC060914701462F50E0CA01B0
:102030000196880F991FE091FC02F091FD02E80FD4
:10204000F91F85919491892B19F48EE991E12BC0A8
:10205000E0910703F0910803208131814150504005
:1020600037FF0CC081E090E002C0880F991F4A95AD
:10207000E2F72070307F822B932B09C081E090E043
:1020800002C0880F991F4A95E2F782279327918310
:102090008083E091FE02F091FF02862F099584E093
:1020A00009C08DEC92E19093F8028093F70281E0F1
:1020B00001C080E01F9108958230D1F0833020F478
:1020C000813009F060C006C0833091F1833809F097
:1020D0005AC05BC080931B02E0910703F091080394
:1020E000608171818091FC029091FD0241E049C0C4
:1020F00080911B028F5F80931B022091FC02309124
:10210000FD02E82FF0E0EE0FFF1FE20FF31F8591B5
:102110009491892B19F481E080931B02E0910703CD
:10212000F091080360817181C90140911B0229C0AF
:10213000A091FC02B091FD0240911B02242F30E0DF
:10214000F9013196EE0FFF1FEA0FFB1F8591949165
:10215000892B19F48EE991E11AC0E0910703F091FF
:1021600008032150304061E070E002C0660F771F25
:102170002A95E2F7808191816827792771836083AE
:10218000CD010E941D0F80E008958DEC92E19093A7
:10219000F8028093F702E0910703F0910803808131
:1021A00091819F70892B21F481E090E0918380835D
:1021B000609137017091380184E090E00E94551BD6
:1021C00081E00895813031F48091FB028F3768F40B
:1021D0008F5F07C0823049F48091FB02882329F089
:1021E00081508093FB020E94980980E090E19093D7
:1021F0003601809335010895823061F0833020F4F8
:10220000813009F054C012C08330D9F0843009F015
:102210004EC032C0809160028D7F8093600282E068
:1022200090E0909332018093310141C0809160022F
:1022300082608093600281E090E09093320180930D
:1022400031018091600282FF09C080915D0290910E
:102250005E0290935A028093590204C010925A026F
:102260001092590280913101909132018B7F9093AD
:1022700032018093310119C08091600282FF08C051
:1022800010925A0210925902809160028B7F0BC00B
:1022900080915D0290915E0290935A028093590260
:1022A000809160028460809360020E945314809148
:1022B0006002209131013091320182FF02C028601A
:1022C00001C0277F3093320120933101089581307E
:1022D00041F4809160028E7F8093600281E090E003
:1022E00009C0823061F48091600281608093600255
:1022F00082E090E09093300180932F0113C08330EF
:1023000069F488E592E09093F0028093EF0282E016
:1023100090E068E572E00E94551B04C0843011F41F
:102320000E94BD1980912F019091300183709070AF
:1023300090639093300180932F0108951F93182F7D
:102340008230D9F0833018F4813081F505C08330B4
:1023500079F1833859F518C10E9485091093480115
:102360008091EE0280FF03C080E695E002C084E722
:1023700095E060E070E041E017C0809148018F5F18
:1023800080934801893018F081E080934801809162
:10239000EE0280FF03C080E695E002C084E795E08E
:1023A00060E070E0409148010E941D0F80E0F3C0A2
:1023B00080914801843009F477C0853048F4823038
:1023C000C9F1833008F056C0813009F0E3C00DC078
:1023D000863009F495C0863008F482C0873009F44D
:1023E000ABC0883009F0D6C0C3C080E99FE09093AD
:1023F000F8028093F7028091EE0280FF03C088EB21
:1024000095E002C086EC95E09093FD028093FC027B
:102410008FE291E0909308038093070380912F014E
:102420009091300190639093300180932F0187E663
:1024300091E11BC080E99FE09093F8028093F7023E
:102440008091EE0280FF03C084ED95E002C082EE31
:1024500095E09093FD028093FC0281E391E09093DC
:102460000803809307038CEF90E19093FF02809321
:10247000FE0290C08CE590E19093F8028093F70201
:102480008091EE0280FF03C088E895E002C080EAF8
:1024900095E09093FD028093FC0287E391E0909396
:1024A00008038093070376C080E99FE09093F802C9
:1024B0008093F7028091EE0280FF03C080EF95E0E9
:1024C00002C08AEF95E09093FD028093FC0280E0C9
:1024D00093E0909308038093070387EF9BE0C5CFB9
:1024E00080E99FE09093F8028093F7028091EE02DA
:1024F00080FF03C084E096E0E6CF8EE096E0E3CF75
:1025000080E99FE09093F8028093F7028091EE02B9
:1025100080FF03C088E196E002C082E296E09093DB
:10252000FD028093FC0283E391E090930803809383
:10253000070382E09CE099CF80E99FE09093F80246
:102540008093F7028091EE0280FF03C08CE296E058
:1025500002C086E396E09093FD028093FC0285E33F
:1025600091E0909308038093070382EE90E17DCF82
:1025700080E090E06091EE020E94471B81E090E0D5
:102580006091FB020E94471B8DEC92E19093F80250
:102590008093F70281E01F910895863040F48430E3
:1025A00038F5813008F47DC0833038F011C08930AF
:1025B000C1F0833809F075C076C00E9498090E9466
:1025C000E20D81E00E94290E8FEF0E94180B69C076
:1025D00080911C0291E0892780931C0284E68093FD
:1025E000020180911C02882309F058C083E057C083
:1025F00080916803853160F08091600281FD08C0A0
:102600000E94010F8091600280618093600244C04B
:102610008091600284FF06C0809160028F7E80936B
:102620006002CBCF0E94230D0E94940C0E94770D74
:102630008091600281FF1CC08091B6039091B70326
:1026400064E040E20E946D0C8091600283FF24C030
:102650000E94C61828E631E0A901481B590BCA019F
:102660000E94290CE82FF0E0E75CFE4F808112C049
:1026700080918E0390918F0364E040E20E946D0C84
:102680008091600283FF08C080918E0390918F0338
:102690000E94290C0E94180B0E94330D80E00E94BA
:1026A000290E80E0089585E00E94290E8EE991E1CF
:1026B0009093F8028093F70281E00895EF92FF92E1
:1026C0000F931F93809166038F5F809366038C3313
:1026D00090F010926603809186038F5F809386034B
:1026E0008C3348F01092860380916703833618F488
:1026F0008F5F8093670380918903833008F45FC004
:10270000E0904A01F0904B0100914C0110914D0175
:102710000894E11CF11C011D111DE0924A01F09288
:102720004B0100934C0110934D0190916803992344
:1027300081F184E6989FC001112464E270E00E9458
:102740009F1A80911D0290911E02680F791F40917F
:1027500085032091690330916A0380918C039091E5
:102760008D0307C0413011F42F5F3F4F685E734007
:10277000019653E0683E7507A8F730936A032093EB
:10278000690380938C0390938D0370931E02609372
:102790001D0260918C0370918D03882777FD8095D1
:1027A000982F20E13EE040E050E00E94741AA8011A
:1027B00097010E94C61A30939503209394031F91AA
:1027C0000F91FF90EF900895FC0109C03196861794
:1027D00031F4415021F48081861731F403C08081A7
:1027E0008823A1F7E0E0F0E0CF010895CF93DF93D5
:1027F000FC01EC0121963091490130518181380F63
:1028000080812AE0829FC0011124380F38310CF0FA
:10281000385137FD385E30937C03FE013196DF017D
:1028200011962181205189813AE0839FC0011124B2
:10283000280F20937D0312962C9112972051119608
:102840008C91839FC0011124280F20937E03DF9178
:10285000CF910895FC01AC014F5F5F4F2181205162
:1028600080813AE0839FC0011124280F20937F03C9
:10287000FA013196DF01119621812051FA018181FF
:10288000839FC0011124280F2093800312962C915E
:102890001297205111968C91839FC0011124280F0B
:1028A0002093810308956091590270915A028BE63A
:1028B00093E00E94691980916B0390916C03A09141
:1028C0006D03B0916E0380939E0390939F03A0933A
:1028D000A003B093A10380916F0390917003A09126
:1028E0007103B09172038093A2039093A303A0930A
:1028F000A403B093A5030895809110038D3409F0CB
:1029000049C08CE093E06CE241E00E94E413009740
:1029100011F00E94F6138CE093E06CE243E00E9419
:10292000E413FC01009711F13297808132968134D3
:10293000E9F4CF010E94121760936F037093700344
:1029400080937103909372038CE093E06CE245E016
:102950000E94E413009751F00E94121760936B03DA
:1029600070936C0380936D0390936E038CE093E0FF
:102970006CE249E00E94E413009711F00E942A14CF
:10298000A6E7B3E0ECE7F3E086E001900D9281501A
:10299000E1F70895873409F077C08CE093E06CE2AA
:1029A00047E00E94E4130E94031B809389038CE09C
:1029B00093E06CE249E00E94E413009789F00E94E2
:1029C000031B90938303809382031816190644F027
:1029D000809121029091220290938303809382033D
:1029E00080918903843008F4C7C1409182035091DB
:1029F00083035093740340937303809187039091F2
:102A000088038417950724F4509388034093870321
:102A10008091210290912202892B21F4509322026D
:102A20004093210220912102309122022417350780
:102A30009CF480918A0390918B03840F951F821BD5
:102A4000930B90938B0380938A03509322024093BD
:102A50002102109285030895421753070CF08CC190
:102A60008091910390919203280F391F241B350BFD
:102A700030939203209391035093220240932102BA
:102A800081E080938503089580910F03863509F0D6
:102A900073C1459A8CE093E06CE241E00E94E4133C
:102AA0000E94031B90938F0380938E038CE093E02E
:102AB0006CE247E00E94E4130E94031B282F8091E0
:102AC0009303821710F42093930380916803882363
:102AD00019F4222309F445C1209368038091600210
:102AE000886080936002809120028F5F8093200233
:102AF000222311F4109220026091EF027091F002F3
:102B000089E26736780720F58091600280FF20C057
:102B10008091200290E083709070892BC9F42093FB
:102B200075038BE693E00E943E19813041F4609179
:102B3000EF027091F00282E090E00E94551B8091BC
:102B4000EF029091F00201969093F0028093EF02D1
:102B50008091600281FF0AC180916B0390916C03A8
:102B6000A0916D03B0916E038093960390939703A9
:102B7000A0939803B093990380916F039091700391
:102B8000A0917103B091720380939A0390939B0379
:102B9000A0939C03B0939D0386E993E00E949F1746
:102BA0002091B6033091B7034091B8035091B90317
:102BB00080914F0190915001A0915101B09152012B
:102BC00082179307A407B5074CF020934F01309369
:102BD000500140935101509352014EC080914E01DB
:102BE000815080934E01882309F049C080915D0295
:102BF00090915E0224E0969587952A95E1F780935F
:102C00001F022091600290E04091590250915A02B7
:102C100022FF03C0481B590B02C0480F591F509395
:102C20005A024093590220915D0230915E028091D8
:102C3000590290915A022817390750F48091600286
:102C400082FD02C020E030E030935A022093590206
:102C50001092B6031092B7031092B8031092B90302
:102C60008FE097E2A0E0B0E080934F019093500195
:102C7000A0935101B09352018EE180934E01809157
:102C8000B6039091B703A091B803B091B903C2976E
:102C9000A105B1050CF06AC08FE097E2A0E0B0E0BA
:102CA00080934F0190935001A0935101B093520132
:102CB0008091600282FF06C08091590290915A0271
:102CC000892B79F08091600282FD17C02091590212
:102CD00030915A0280915D0290915E022817390767
:102CE00060F0809160028D7F8093600282E090E0CE
:102CF000909332018093310139C0809160024091FC
:102D0000590250915A0282FF03C04150504002C004
:102D10004F5F5F4F50935A02409359020E945314E1
:102D20008091960390919703A0919803B091990395
:102D300080936B0390936C03A0936D03B0936E0329
:102D400080919A0390919B03A0919C03B0919D0365
:102D500080936F0390937003A0937103B0937203F9
:102D600005C080916002877F809360020E945E139D
:102D700085E08093610245980895AF92BF92CF920B
:102D8000DF92EF92FF920F931F93E12CF12C012D14
:102D9000F0E41F2F07C0E2E016950795F794E7943B
:102DA000EA95D1F76E157F0580079107A0F35B01C7
:102DB0006C0120E030E040E050E024C0DA01C901BD
:102DC0008E0D9F1DA01FB11FA816B906CA06DB06EF
:102DD00070F0A81AB90ACA0ADB0AD801C701880F1D
:102DE000991FAA1FBB1F280F391F4A1F5B1F56952B
:102DF00047953795279582E016950795F794E794C0
:102E00008A95D1F7E114F10401051105B9F6B9016C
:102E1000CA011F910F91FF90EF90DF90CF90BF906C
:102E2000AF9008958F929F92AF92BF92CF92DF9210
:102E3000EF92FF920F931F93CF93DF93EC01FC016E
:102E400001C031969E2E9C1A80818C32D1F7882445
:102E5000A1E0AA2EB12CC12CD12CEE24FF24870195
:102E60009A94FE01E90DF11D80818E3209F49A9445
:102E7000FE01E90DF11D608170E06053704088270C
:102E800077FD8095982FA60195010E94741AE60E91
:102E9000F71E081F191F8394C601B5012AE030E010
:102EA00040E050E00E94741A5B016C0186E08816D5
:102EB000B9F6C801B70126E030E040E050E00E94DA
:102EC000E81AC901DA017C018D01C601B5012AE0C9
:102ED00030E040E050E00E94E81A59016A011EC04B
:102EE0009A94FE01E90DF11D608170E0605370401D
:102EF000882777FD8095982F9501A6010E94741A66
:102F0000E60EF71E081F191FB501C6012AE030E0C2
:102F100040E050E00E94741A5B016C01992001F7B7
:102F2000B701C801DF91CF911F910F91FF90EF90F2
:102F3000DF90CF90BF90AF909F908F9008956F9249
:102F40007F928F929F92AF92BF92CF92DF92EF9239
:102F5000FF920F931F93CF93DF93EC012C853D8558
:102F60004E855F859A01552737FD5095452F8C81F9
:102F70009D81AE81BF81CD01BB2797FDB095AB2F61
:102F8000820F931F97FF03C0909581959F4F63E039
:102F900070E00E94B31A6B3528F080E090E0A0E06A
:102FA000B0E010C0E62FF0E0EE0FFF1FED5AFE4F2D
:102FB00080819181A0E0B0E0673320F4880F991FF1
:102FC000AA1FBB1F888B998BAA8BBB8B2885398541
:102FD0004A855B8588819981AA81BB81281B390B31
:102FE0004A0B5B0BAC84BD84CE84DF848C819D81D5
:102FF000AE81BF81A81AB90ACA0ADB0A57FD0BC005
:10300000D7FC03C07FEF6FE010C0211531054105EB
:10301000510549F405C0D7FC03C071E068E005C064
:103020007FEF67E002C071E060E0C90137FF03C0D5
:10303000909581959F4F7C010027F7FC0095102FFC
:10304000C501B7FE03C0909581959F4F3C01882430
:1030500077FC8094982CD401C301880F991FAA1F74
:10306000BB1FE816F9060A071B07F4F4D801C701CD
:10307000880F991FAA1FBB1F681679068A069B0630
:1030800034F083E0789FC0011124680F0DC06E14E6
:103090007F048006910614F0770F05C0E614F7044C
:1030A000080519050CF0670F6EA32EEBE21626E952
:1030B000F20620E0020720E0120748F48EEB6816C3
:1030C00086E9780680E0880680E0980618F08FEFA1
:1030D0008FA345C0288939894A895B89C801B7010E
:1030E0000E94741A20EA36E841E050E00E94E81A93
:1030F00059016A01288F398F4A8F5B8FC401B30150
:1031000024EC32EB41E050E00E94741A20EA36E8E9
:1031100041E050E00E94E81A2C8F3D8F4E8F5F8F68
:10312000B901CA010E94741A7B018C01C601B50164
:10313000A60195010E94741AE60EF71E081F191FBA
:10314000C801B7010E94BD1680E090E068A379A392
:103150008AA39BA3605177428040904044F08FE067
:1031600097E2A0E0B0E088A399A3AAA3BBA3DF9154
:10317000CF911F910F91FF90EF90DF90CF90BF9074
:10318000AF909F908F907F906F9008958091BC0337
:1031900090E00C968F70907026E130E0AC01429F79
:1031A000C001439F900D529F900D112420918E03DA
:1031B00030918F03281B390B37FF02C028593E4F2F
:1031C000C9010895429887ED8EBD0DB407FEFDCF6D
:1031D0001EBC0DB407FEFDCF0EB407FEF9CF429A18
:1031E00042980895EF92FF920F931F93F82EE92EC5
:1031F000062F142F0E94E21884E88EBD0DB407FE3E
:10320000FDCF1EBC0DB407FEFDCF1EBC0DB407FEE6
:10321000FDCF0EBD0DB407FEFDCF8F2D9E2D9C0161
:10322000F90107C080818EBD0DB407FEFDCF319638
:1032300011501123B9F7429A1F910F91FF90EF900F
:103240000895FF920F931F93F82E092F162F0E94B7
:10325000E2181EBD0DB407FEFDCF0EBD0DB407FE76
:10326000FDCFFEBC0DB407FEFDCF1EBC0DB407FEA6
:10327000FDCF429A1F910F91FF9008951F93CF9316
:10328000DF939C01EB0185E761327807E8F4CB011D
:103290006FE070E00E949F1A182F61E1869FB001D5
:1032A0001124C90141E10E94F2181E3068F0CE01DC
:1032B0006FE070E00E949F1ACB01880F991F63E8AE
:1032C0000E94211981E001C080E0DF91CF911F9120
:1032D0000895EF92FF920F931F93CF93DF938C018A
:1032E0007B01CB016FE070E00E949F1AEB0180919F
:1032F000090290910A026817790751F0CB01880FF3
:10330000991F65E50E942119D0930A02C093090212
:103310000E94E21886ED8EBD0DB407FEFDCF1EBCE7
:103320000DB407FEFDCF1EBC0DB407FEFDCFC701D7
:103330006FE070E00E949F1A91E1899FC001112403
:103340008EBD0DB407FEFDCF1EBC0DB407FEFDCF34
:1033500091E11EBC0DB407FEFDCF8EB5F801808350
:10336000915019F00F5F1F4FF4CF429ADF91CF9128
:103370001F910F91FF90EF900895FF920F931F936D
:10338000CF93DF938091EF029091F0026FE070E0B5
:103390000E949F1ACB01880F991F63E80E94211990
:1033A0008091EF029091F0028855924009F44FC04D
:1033B00062EF71E00E94B31AF62EF394C8E5D2E0F2
:1033C00000E010E017C0CE016F2D70E00E94B31A2C
:1033D000892B19F0C217D30761F486E993E0BE0187
:1033E0000E94691986E993E0B8010E943E190F5FB7
:1033F0001F4F21962091EF023091F0022C173D07CC
:1034000010F7C8016FE070E00E94B31ACB01880F7B
:10341000991F63E80E9421198091EF029091F002B8
:103420006FE070E00E949F1ACB01880F991F63E53F
:103430000E94211910925A021092590210935E02B2
:1034400000935D02809160028D7F80936002DF9126
:10345000CF911F910F91FF9008950F931F93CF93DA
:10346000DF938C01EB0120E160307207C0F50E9410
:10347000E218C0FD02C090E001C090E882ED8EBD70
:103480000DB407FEFDCFDEBD0DB407FEFDCFFE017E
:10349000EE7FEEBD0DB407FEFDCF9EBD0DB407FE61
:1034A000FDCF1EBC0DB407FEFDCF1EBC0DB407FE44
:1034B000FDCF1EBC0DB407FEFDCF1EBC0DB407FE34
:1034C000FDCF90E81EBC0DB407FEFDCF8EB5F80110
:1034D0008083915019F00F5F1F4FF4CF429ADF9114
:1034E000CF911F910F910895629FD001739FF001BA
:1034F000829FE00DF11D649FE00DF11D929FF00D84
:10350000839FF00D749FF00D659FF00D9927729FBA
:10351000B00DE11DF91F639FB00DE11DF91FBD0145
:10352000CF0111240895991B79E004C0991F9617C3
:1035300008F0961B881F7A95C9F780950895AA1BF5
:10354000BB1B51E107C0AA1FBB1FA617B70710F08E
:10355000A61BB70B881F991F5A95A9F780959095C0
:10356000BC01CD01089597FB092E07260AD077FDEF
:1035700004D0E5DF06D000201AF4709561957F4FE6
:103580000895F6F7909581959F4F0895A1E21A2E20
:10359000AA1BBB1BFD010DC0AA1FBB1FEE1FFF1FF7
:1035A000A217B307E407F50720F0A21BB30BE40B47
:1035B000F50B661F771F881F991F1A9469F760958E
:1035C0007095809590959B01AC01BD01CF01089548
:1035D00097FB092E05260ED057FD04D0D7DF0AD061
:1035E000001C38F450954095309521953F4F4F4F32
:1035F0005F4F0895F6F790958095709561957F4F90
:103600008F4F9F4F0895FC0188279927E8942191B7
:103610002032E9F3293010F02E30C8F32B3241F07C
:103620002D3239F4689404C00E94311B820F911D21
:10363000219120532A30C0F31EF4909581959F4F1D
:103640000895FB01DC0105900D920020E1F708953B
:10365000FB01DC0102C001900D9241505040D8F7AF
:1036600008957AE0979F902D879F802D910D1124CA
:103670000895F999FECF92BD81BDF89A992780B53A
:103680000895A8E1B0E042E050E00C945C1B262FC6
:10369000F999FECF1FBA92BD81BD20BD0FB6F89437
:1036A000FA9AF99A0FBE019608950E94471B272F98
:1036B0000C94481BDC01CB01FC01F999FECF06C03C
:1036C000F2BDE1BDF89A319600B40D9241505040E0
:0836D000B8F70895F894FFCF4C
:1036D8005AFF64FF2055534220002020202000522A
:1036E8004F55544500545241434B0053544F5020BA
:1036F800004B4D2F48004D2F482000563132000214
:1037080030020000200010550000070605040302DF
:1037180007002030383C3E010101010000001E0F67
:1037280027000062D95AD940D916D9DAD88ED831AB
:10373800D8C3D744D7B5D615D664D5A2D4D0D3ED3F
:10374800D2FAD1F6D0E2CFBECE8ACD46CCF2CA8E1E
:10375800C91AC897C604C562C3B1C1F0BF21BE4328
:10376800BC56BA5AB850B638B412B2DEAF9CAD4D9A
:10377800ABF1A887A610A48CA1FC9E609CB7990207
:1037880097429476919E8EBC8BCE88D685D4828EB5
:10379800FF61F920F3CCEC66E6EDDF64D9C9D21EEF
:1037A800CC63C599BEBFB7D8B0E2A9E0A2D09BB59B
:1037B800948E8D5C861F7FD97789703069CF616759
:1037C8005AF852824B0644853CFF34752DE725573D
:0C37D8001EC4162F0F99070300FFFF000E
:00000001FF
